
C:\Documents and Settings\jarek\Pulpit\Privet\Magisterka\Programy\1\um0427\FWLib\project\RIDE\STM3210E-EVAL\t6963c_graf.o:     file format elf32-littlearm
C:\Documents and Settings\jarek\Pulpit\Privet\Magisterka\Programy\1\um0427\FWLib\project\RIDE\STM3210E-EVAL\t6963c_graf.o

Disassembly of section .text.GLCD_Obraz:

00000000 <GLCD_Obraz>:
GLCD_Obraz():
C:\Documents and Settings\jarek\Pulpit\Privet\Magisterka\Programy\1\um0427\FWLib\project/t6963c_graf.c:110
   0:	b570      	push	{r4, r5, r6, lr}
C:\Documents and Settings\jarek\Pulpit\Privet\Magisterka\Programy\1\um0427\FWLib\project/t6963c_graf.c:113
   2:	2428      	movs	r4, #40
   4:	fb01 f104 	mul.w	r1, r1, r4
C:\Documents and Settings\jarek\Pulpit\Privet\Magisterka\Programy\1\um0427\FWLib\project/t6963c_graf.c:110
   8:	4606      	mov	r6, r0
C:\Documents and Settings\jarek\Pulpit\Privet\Magisterka\Programy\1\um0427\FWLib\project/t6963c_graf.c:113
   a:	f501 6080 	add.w	r0, r1, #1024	; 0x400
C:\Documents and Settings\jarek\Pulpit\Privet\Magisterka\Programy\1\um0427\FWLib\project/t6963c_graf.c:110
   e:	4615      	mov	r5, r2
C:\Documents and Settings\jarek\Pulpit\Privet\Magisterka\Programy\1\um0427\FWLib\project/t6963c_graf.c:113
  10:	f7ff fffe 	bl	0 <GLCD_Ustaw_Adres>
C:\Documents and Settings\jarek\Pulpit\Privet\Magisterka\Programy\1\um0427\FWLib\project/t6963c_graf.c:114
  14:	20b0      	movs	r0, #176
C:\Documents and Settings\jarek\Pulpit\Privet\Magisterka\Programy\1\um0427\FWLib\project/t6963c_graf.c:115
  16:	fb05 f504 	mul.w	r5, r5, r4
C:\Documents and Settings\jarek\Pulpit\Privet\Magisterka\Programy\1\um0427\FWLib\project/t6963c_graf.c:114
  1a:	f7ff fffe 	bl	0 <GLCD_Write_Command>
C:\Documents and Settings\jarek\Pulpit\Privet\Magisterka\Programy\1\um0427\FWLib\project/t6963c_graf.c:115
  1e:	2400      	movs	r4, #0
  20:	e003      	b.n	2a <GLCD_Obraz+0x2a>
C:\Documents and Settings\jarek\Pulpit\Privet\Magisterka\Programy\1\um0427\FWLib\project/t6963c_graf.c:116
  22:	57a0      	ldrsb	r0, [r4, r6]
  24:	f7ff fffe 	bl	0 <GLCD_Write_Data>
C:\Documents and Settings\jarek\Pulpit\Privet\Magisterka\Programy\1\um0427\FWLib\project/t6963c_graf.c:115
  28:	3401      	adds	r4, #1
  2a:	42ac      	cmp	r4, r5
  2c:	dbf9      	blt.n	22 <GLCD_Obraz+0x22>
C:\Documents and Settings\jarek\Pulpit\Privet\Magisterka\Programy\1\um0427\FWLib\project/t6963c_graf.c:118
  2e:	20b2      	movs	r0, #178
  30:	f7ff fffe 	bl	0 <GLCD_Write_Command>
C:\Documents and Settings\jarek\Pulpit\Privet\Magisterka\Programy\1\um0427\FWLib\project/t6963c_graf.c:119
  34:	bd70      	pop	{r4, r5, r6, pc}
  36:	46c0      	nop			(mov r8, r8)
Disassembly of section .text.GLCD_Kolo:

00000000 <GLCD_Kolo>:
GLCD_Kolo():
C:\Documents and Settings\jarek\Pulpit\Privet\Magisterka\Programy\1\um0427\FWLib\project/t6963c_graf.c:65
   0:	e92d 4ff7 	stmdb	sp!, {r0, r1, r2, r4, r5, r6, r7, r8, r9, sl, fp, lr}
   4:	4698      	mov	r8, r3
C:\Documents and Settings\jarek\Pulpit\Privet\Magisterka\Programy\1\um0427\FWLib\project/t6963c_graf.c:70
   6:	0053      	lsls	r3, r2, #1
C:\Documents and Settings\jarek\Pulpit\Privet\Magisterka\Programy\1\um0427\FWLib\project/t6963c_graf.c:65
   8:	9001      	str	r0, [sp, #4]
   a:	468b      	mov	fp, r1
C:\Documents and Settings\jarek\Pulpit\Privet\Magisterka\Programy\1\um0427\FWLib\project/t6963c_graf.c:70
   c:	f1c3 0a03 	rsb	sl, r3, #3	; 0x3
  10:	4617      	mov	r7, r2
  12:	f04f 0900 	mov.w	r9, #0	; 0x0
C:\Documents and Settings\jarek\Pulpit\Privet\Magisterka\Programy\1\um0427\FWLib\project/t6963c_graf.c:71
  16:	e04a      	b.n	ae <GLCD_Kolo+0xae>
C:\Documents and Settings\jarek\Pulpit\Privet\Magisterka\Programy\1\um0427\FWLib\project/t6963c_graf.c:65
  18:	9b01      	ldr	r3, [sp, #4]
C:\Documents and Settings\jarek\Pulpit\Privet\Magisterka\Programy\1\um0427\FWLib\project/t6963c_graf.c:73
  1a:	eb07 060b 	add.w	r6, r7, fp
C:\Documents and Settings\jarek\Pulpit\Privet\Magisterka\Programy\1\um0427\FWLib\project/t6963c_graf.c:65
  1e:	eb09 0403 	add.w	r4, r9, r3
C:\Documents and Settings\jarek\Pulpit\Privet\Magisterka\Programy\1\um0427\FWLib\project/t6963c_graf.c:73
  22:	4620      	mov	r0, r4
  24:	4631      	mov	r1, r6
C:\Documents and Settings\jarek\Pulpit\Privet\Magisterka\Programy\1\um0427\FWLib\project/t6963c_graf.c:74
  26:	ebc7 050b 	rsb	r5, r7, fp
C:\Documents and Settings\jarek\Pulpit\Privet\Magisterka\Programy\1\um0427\FWLib\project/t6963c_graf.c:73
  2a:	4642      	mov	r2, r8
  2c:	f7ff fffe 	bl	0 <GLCD_SetPixel>
C:\Documents and Settings\jarek\Pulpit\Privet\Magisterka\Programy\1\um0427\FWLib\project/t6963c_graf.c:74
  30:	4620      	mov	r0, r4
  32:	4629      	mov	r1, r5
  34:	4642      	mov	r2, r8
  36:	f7ff fffe 	bl	0 <GLCD_SetPixel>
  3a:	9b01      	ldr	r3, [sp, #4]
C:\Documents and Settings\jarek\Pulpit\Privet\Magisterka\Programy\1\um0427\FWLib\project/t6963c_graf.c:75
  3c:	4631      	mov	r1, r6
C:\Documents and Settings\jarek\Pulpit\Privet\Magisterka\Programy\1\um0427\FWLib\project/t6963c_graf.c:74
  3e:	ebc9 0403 	rsb	r4, r9, r3
C:\Documents and Settings\jarek\Pulpit\Privet\Magisterka\Programy\1\um0427\FWLib\project/t6963c_graf.c:75
  42:	4620      	mov	r0, r4
  44:	4642      	mov	r2, r8
  46:	f7ff fffe 	bl	0 <GLCD_SetPixel>
C:\Documents and Settings\jarek\Pulpit\Privet\Magisterka\Programy\1\um0427\FWLib\project/t6963c_graf.c:76
  4a:	4620      	mov	r0, r4
  4c:	4629      	mov	r1, r5
  4e:	4642      	mov	r2, r8
  50:	f7ff fffe 	bl	0 <GLCD_SetPixel>
C:\Documents and Settings\jarek\Pulpit\Privet\Magisterka\Programy\1\um0427\FWLib\project/t6963c_graf.c:77
  54:	9b01      	ldr	r3, [sp, #4]
C:\Documents and Settings\jarek\Pulpit\Privet\Magisterka\Programy\1\um0427\FWLib\project/t6963c_graf.c:65
  56:	eb09 060b 	add.w	r6, r9, fp
C:\Documents and Settings\jarek\Pulpit\Privet\Magisterka\Programy\1\um0427\FWLib\project/t6963c_graf.c:77
  5a:	18fc      	adds	r4, r7, r3
  5c:	4620      	mov	r0, r4
  5e:	4631      	mov	r1, r6
  60:	4642      	mov	r2, r8
  62:	ebc9 050b 	rsb	r5, r9, fp
  66:	f7ff fffe 	bl	0 <GLCD_SetPixel>
C:\Documents and Settings\jarek\Pulpit\Privet\Magisterka\Programy\1\um0427\FWLib\project/t6963c_graf.c:78
  6a:	4620      	mov	r0, r4
  6c:	4629      	mov	r1, r5
  6e:	4642      	mov	r2, r8
  70:	f7ff fffe 	bl	0 <GLCD_SetPixel>
C:\Documents and Settings\jarek\Pulpit\Privet\Magisterka\Programy\1\um0427\FWLib\project/t6963c_graf.c:79
  74:	9b01      	ldr	r3, [sp, #4]
  76:	4631      	mov	r1, r6
  78:	1bdc      	subs	r4, r3, r7
  7a:	4620      	mov	r0, r4
  7c:	4642      	mov	r2, r8
  7e:	f7ff fffe 	bl	0 <GLCD_SetPixel>
C:\Documents and Settings\jarek\Pulpit\Privet\Magisterka\Programy\1\um0427\FWLib\project/t6963c_graf.c:80
  82:	4620      	mov	r0, r4
  84:	4629      	mov	r1, r5
  86:	4642      	mov	r2, r8
  88:	f7ff fffe 	bl	0 <GLCD_SetPixel>
C:\Documents and Settings\jarek\Pulpit\Privet\Magisterka\Programy\1\um0427\FWLib\project/t6963c_graf.c:81
  8c:	f1ba 0f00 	cmp.w	sl, #0	; 0x0
  90:	da04      	bge.n	9c <GLCD_SetPixel+0x9c>
C:\Documents and Settings\jarek\Pulpit\Privet\Magisterka\Programy\1\um0427\FWLib\project/t6963c_graf.c:82
  92:	f10a 0306 	add.w	r3, sl, #6	; 0x6
  96:	eb03 0a89 	add.w	sl, r3, r9, lsl #2
  9a:	e006      	b.n	aa <GLCD_SetPixel+0xaa>
C:\Documents and Settings\jarek\Pulpit\Privet\Magisterka\Programy\1\um0427\FWLib\project/t6963c_graf.c:84
  9c:	ebc7 0309 	rsb	r3, r7, r9
  a0:	f10a 020a 	add.w	r2, sl, #10	; 0xa
  a4:	eb02 0a83 	add.w	sl, r2, r3, lsl #2
  a8:	3f01      	subs	r7, #1
  aa:	f109 0901 	add.w	r9, r9, #1	; 0x1
C:\Documents and Settings\jarek\Pulpit\Privet\Magisterka\Programy\1\um0427\FWLib\project/t6963c_graf.c:71
  ae:	45b9      	cmp	r9, r7
  b0:	ddb2      	ble.n	18 <GLCD_SetPixel+0x18>
C:\Documents and Settings\jarek\Pulpit\Privet\Magisterka\Programy\1\um0427\FWLib\project/t6963c_graf.c:86
  b2:	e8bd 8ffe 	ldmia.w	sp!, {r1, r2, r3, r4, r5, r6, r7, r8, r9, sl, fp, pc}
  b6:	46c0      	nop			(mov r8, r8)
Disassembly of section .text.GLCD_Linia:

00000000 <GLCD_Linia>:
GLCD_Linia():
C:\Documents and Settings\jarek\Pulpit\Privet\Magisterka\Programy\1\um0427\FWLib\project/t6963c_graf.c:5
   0:	e92d 4ff7 	stmdb	sp!, {r0, r1, r2, r4, r5, r6, r7, r8, r9, sl, fp, lr}
   4:	4699      	mov	r9, r3
   6:	9200      	str	r2, [sp, #0]
C:\Documents and Settings\jarek\Pulpit\Privet\Magisterka\Programy\1\um0427\FWLib\project/t6963c_graf.c:10
   8:	1a13      	subs	r3, r2, r0
C:\Documents and Settings\jarek\Pulpit\Privet\Magisterka\Programy\1\um0427\FWLib\project/t6963c_graf.c:11
   a:	ebb9 0201 	subs.w	r2, r9, r1
C:\Documents and Settings\jarek\Pulpit\Privet\Magisterka\Programy\1\um0427\FWLib\project/t6963c_graf.c:5
   e:	4606      	mov	r6, r0
  10:	460d      	mov	r5, r1
  12:	f89d a030 	ldrb.w	sl, [sp, #48]
C:\Documents and Settings\jarek\Pulpit\Privet\Magisterka\Programy\1\um0427\FWLib\project/t6963c_graf.c:11
  16:	d401      	bmi.n	1c <GLCD_Linia+0x1c>
  18:	2101      	movs	r1, #1
  1a:	e002      	b.n	22 <GLCD_Linia+0x22>
C:\Documents and Settings\jarek\Pulpit\Privet\Magisterka\Programy\1\um0427\FWLib\project/t6963c_graf.c:13
  1c:	4252      	negs	r2, r2
  1e:	f04f 31ff 	mov.w	r1, #4294967295	; 0xffffffff
C:\Documents and Settings\jarek\Pulpit\Privet\Magisterka\Programy\1\um0427\FWLib\project/t6963c_graf.c:20
  22:	2b00      	cmp	r3, #0
C:\Documents and Settings\jarek\Pulpit\Privet\Magisterka\Programy\1\um0427\FWLib\project/t6963c_graf.c:13
  24:	9101      	str	r1, [sp, #4]
C:\Documents and Settings\jarek\Pulpit\Privet\Magisterka\Programy\1\um0427\FWLib\project/t6963c_graf.c:20
  26:	db02      	blt.n	2e <GLCD_Linia+0x2e>
  28:	f04f 0b01 	mov.w	fp, #1	; 0x1
  2c:	e002      	b.n	34 <GLCD_Linia+0x34>
C:\Documents and Settings\jarek\Pulpit\Privet\Magisterka\Programy\1\um0427\FWLib\project/t6963c_graf.c:22
  2e:	425b      	negs	r3, r3
  30:	f04f 3bff 	mov.w	fp, #4294967295	; 0xffffffff
C:\Documents and Settings\jarek\Pulpit\Privet\Magisterka\Programy\1\um0427\FWLib\project/t6963c_graf.c:29
  34:	ea4f 0842 	mov.w	r8, r2, lsl #1
C:\Documents and Settings\jarek\Pulpit\Privet\Magisterka\Programy\1\um0427\FWLib\project/t6963c_graf.c:30
  38:	005f      	lsls	r7, r3, #1
C:\Documents and Settings\jarek\Pulpit\Privet\Magisterka\Programy\1\um0427\FWLib\project/t6963c_graf.c:31
  3a:	4630      	mov	r0, r6
  3c:	4629      	mov	r1, r5
  3e:	4652      	mov	r2, sl
  40:	f7ff fffe 	bl	0 <GLCD_SetPixel>
C:\Documents and Settings\jarek\Pulpit\Privet\Magisterka\Programy\1\um0427\FWLib\project/t6963c_graf.c:32
  44:	4547      	cmp	r7, r8
  46:	dd12      	ble.n	6e <GLCD_Linia+0x6e>
C:\Documents and Settings\jarek\Pulpit\Privet\Magisterka\Programy\1\um0427\FWLib\project/t6963c_graf.c:34
  48:	eba8 0467 	sub.w	r4, r8, r7, asr #1
C:\Documents and Settings\jarek\Pulpit\Privet\Magisterka\Programy\1\um0427\FWLib\project/t6963c_graf.c:35
  4c:	e00b      	b.n	66 <GLCD_Linia+0x66>
C:\Documents and Settings\jarek\Pulpit\Privet\Magisterka\Programy\1\um0427\FWLib\project/t6963c_graf.c:37
  4e:	2c00      	cmp	r4, #0
  50:	db02      	blt.n	58 <GLCD_Linia+0x58>
C:\Documents and Settings\jarek\Pulpit\Privet\Magisterka\Programy\1\um0427\FWLib\project/t6963c_graf.c:39
  52:	9a01      	ldr	r2, [sp, #4]
C:\Documents and Settings\jarek\Pulpit\Privet\Magisterka\Programy\1\um0427\FWLib\project/t6963c_graf.c:40
  54:	1be4      	subs	r4, r4, r7
C:\Documents and Settings\jarek\Pulpit\Privet\Magisterka\Programy\1\um0427\FWLib\project/t6963c_graf.c:39
  56:	18ad      	adds	r5, r5, r2
C:\Documents and Settings\jarek\Pulpit\Privet\Magisterka\Programy\1\um0427\FWLib\project/t6963c_graf.c:40
  58:	445e      	add	r6, fp
C:\Documents and Settings\jarek\Pulpit\Privet\Magisterka\Programy\1\um0427\FWLib\project/t6963c_graf.c:44
  5a:	4630      	mov	r0, r6
  5c:	4629      	mov	r1, r5
  5e:	4652      	mov	r2, sl
C:\Documents and Settings\jarek\Pulpit\Privet\Magisterka\Programy\1\um0427\FWLib\project/t6963c_graf.c:43
  60:	4444      	add	r4, r8
C:\Documents and Settings\jarek\Pulpit\Privet\Magisterka\Programy\1\um0427\FWLib\project/t6963c_graf.c:44
  62:	f7ff fffe 	bl	0 <GLCD_SetPixel>
C:\Documents and Settings\jarek\Pulpit\Privet\Magisterka\Programy\1\um0427\FWLib\project/t6963c_graf.c:35
  66:	9b00      	ldr	r3, [sp, #0]
  68:	429e      	cmp	r6, r3
  6a:	d1f0      	bne.n	4e <GLCD_Linia+0x4e>
  6c:	e011      	b.n	92 <GLCD_Linia+0x92>
C:\Documents and Settings\jarek\Pulpit\Privet\Magisterka\Programy\1\um0427\FWLib\project/t6963c_graf.c:49
  6e:	eba7 0468 	sub.w	r4, r7, r8, asr #1
C:\Documents and Settings\jarek\Pulpit\Privet\Magisterka\Programy\1\um0427\FWLib\project/t6963c_graf.c:50
  72:	e00c      	b.n	8e <GLCD_Linia+0x8e>
C:\Documents and Settings\jarek\Pulpit\Privet\Magisterka\Programy\1\um0427\FWLib\project/t6963c_graf.c:55
  74:	9901      	ldr	r1, [sp, #4]
C:\Documents and Settings\jarek\Pulpit\Privet\Magisterka\Programy\1\um0427\FWLib\project/t6963c_graf.c:52
  76:	2c00      	cmp	r4, #0
C:\Documents and Settings\jarek\Pulpit\Privet\Magisterka\Programy\1\um0427\FWLib\project/t6963c_graf.c:54
  78:	bfa4      	itt	ge
  7a:	445e      	addge	r6, fp
C:\Documents and Settings\jarek\Pulpit\Privet\Magisterka\Programy\1\um0427\FWLib\project/t6963c_graf.c:55
  7c:	ebc8 0404 	rsbge	r4, r8, r4
  80:	186d      	adds	r5, r5, r1
C:\Documents and Settings\jarek\Pulpit\Privet\Magisterka\Programy\1\um0427\FWLib\project/t6963c_graf.c:59
  82:	4630      	mov	r0, r6
  84:	4629      	mov	r1, r5
  86:	4652      	mov	r2, sl
C:\Documents and Settings\jarek\Pulpit\Privet\Magisterka\Programy\1\um0427\FWLib\project/t6963c_graf.c:58
  88:	19e4      	adds	r4, r4, r7
C:\Documents and Settings\jarek\Pulpit\Privet\Magisterka\Programy\1\um0427\FWLib\project/t6963c_graf.c:59
  8a:	f7ff fffe 	bl	0 <GLCD_SetPixel>
C:\Documents and Settings\jarek\Pulpit\Privet\Magisterka\Programy\1\um0427\FWLib\project/t6963c_graf.c:50
  8e:	454d      	cmp	r5, r9
  90:	d1f0      	bne.n	74 <GLCD_SetPixel+0x74>
C:\Documents and Settings\jarek\Pulpit\Privet\Magisterka\Programy\1\um0427\FWLib\project/t6963c_graf.c:62
  92:	e8bd 8ffe 	ldmia.w	sp!, {r1, r2, r3, r4, r5, r6, r7, r8, r9, sl, fp, pc}
  96:	46c0      	nop			(mov r8, r8)
Disassembly of section .text.GLCD_Kwadrat_Wypelniony:

00000000 <GLCD_Kwadrat_Wypelniony>:
GLCD_Kwadrat_Wypelniony():
C:\Documents and Settings\jarek\Pulpit\Privet\Magisterka\Programy\1\um0427\FWLib\project/t6963c_graf.c:99
   0:	e92d 41f3 	stmdb	sp!, {r0, r1, r4, r5, r6, r7, r8, lr}
   4:	4680      	mov	r8, r0
   6:	4617      	mov	r7, r2
   8:	461e      	mov	r6, r3
   a:	f89d 5020 	ldrb.w	r5, [sp, #32]
   e:	460c      	mov	r4, r1
C:\Documents and Settings\jarek\Pulpit\Privet\Magisterka\Programy\1\um0427\FWLib\project/t6963c_graf.c:102
  10:	e007      	b.n	22 <GLCD_Kwadrat_Wypelniony+0x22>
C:\Documents and Settings\jarek\Pulpit\Privet\Magisterka\Programy\1\um0427\FWLib\project/t6963c_graf.c:104
  12:	4621      	mov	r1, r4
  14:	4623      	mov	r3, r4
  16:	4640      	mov	r0, r8
  18:	463a      	mov	r2, r7
  1a:	9500      	str	r5, [sp, #0]
  1c:	f7ff fffe 	bl	0 <GLCD_Kwadrat_Wypelniony>
C:\Documents and Settings\jarek\Pulpit\Privet\Magisterka\Programy\1\um0427\FWLib\project/t6963c_graf.c:102
  20:	3401      	adds	r4, #1
  22:	42b4      	cmp	r4, r6
  24:	ddf5      	ble.n	12 <GLCD_Kwadrat_Wypelniony+0x12>
C:\Documents and Settings\jarek\Pulpit\Privet\Magisterka\Programy\1\um0427\FWLib\project/t6963c_graf.c:106
  26:	e8bd 81fc 	ldmia.w	sp!, {r2, r3, r4, r5, r6, r7, r8, pc}
  2a:	46c0      	nop			(mov r8, r8)
Disassembly of section .text.GLCD_Kwadrat:

00000000 <GLCD_Kwadrat>:
GLCD_Kwadrat():
C:\Documents and Settings\jarek\Pulpit\Privet\Magisterka\Programy\1\um0427\FWLib\project/t6963c_graf.c:89
   0:	e92d 4373 	stmdb	sp!, {r0, r1, r4, r5, r6, r8, r9, lr}
   4:	f89d 4020 	ldrb.w	r4, [sp, #32]
   8:	461d      	mov	r5, r3
   a:	4681      	mov	r9, r0
   c:	4690      	mov	r8, r2
C:\Documents and Settings\jarek\Pulpit\Privet\Magisterka\Programy\1\um0427\FWLib\project/t6963c_graf.c:90
   e:	460b      	mov	r3, r1
C:\Documents and Settings\jarek\Pulpit\Privet\Magisterka\Programy\1\um0427\FWLib\project/t6963c_graf.c:89
  10:	460e      	mov	r6, r1
C:\Documents and Settings\jarek\Pulpit\Privet\Magisterka\Programy\1\um0427\FWLib\project/t6963c_graf.c:90
  12:	9400      	str	r4, [sp, #0]
  14:	f7ff fffe 	bl	0 <GLCD_Kwadrat>
C:\Documents and Settings\jarek\Pulpit\Privet\Magisterka\Programy\1\um0427\FWLib\project/t6963c_graf.c:91
  18:	4648      	mov	r0, r9
  1a:	4629      	mov	r1, r5
  1c:	4642      	mov	r2, r8
  1e:	462b      	mov	r3, r5
  20:	9400      	str	r4, [sp, #0]
  22:	f7ff fffe 	bl	0 <GLCD_Kwadrat>
C:\Documents and Settings\jarek\Pulpit\Privet\Magisterka\Programy\1\um0427\FWLib\project/t6963c_graf.c:92
  26:	4640      	mov	r0, r8
  28:	4631      	mov	r1, r6
  2a:	4642      	mov	r2, r8
  2c:	462b      	mov	r3, r5
  2e:	9400      	str	r4, [sp, #0]
  30:	f7ff fffe 	bl	0 <GLCD_Kwadrat>
C:\Documents and Settings\jarek\Pulpit\Privet\Magisterka\Programy\1\um0427\FWLib\project/t6963c_graf.c:93
  34:	4648      	mov	r0, r9
  36:	4631      	mov	r1, r6
  38:	464a      	mov	r2, r9
  3a:	462b      	mov	r3, r5
  3c:	9400      	str	r4, [sp, #0]
  3e:	f7ff fffe 	bl	0 <GLCD_Kwadrat>
C:\Documents and Settings\jarek\Pulpit\Privet\Magisterka\Programy\1\um0427\FWLib\project/t6963c_graf.c:94
  42:	e8bd 837c 	ldmia.w	sp!, {r2, r3, r4, r5, r6, r8, r9, pc}
  46:	46c0      	nop			(mov r8, r8)
